:020000000628D0
:080008000B110900831685109D
:1000100083120130A200AA2081200130A200AA2070
:100020000130003C031952282030A4004030240243
:10003000013003180001003C031923282408910013
:100040006120A40A16280130A200AA200030A400D2
:1000500010302402013003180001003C0319382835
:1000600001309E008820C8308E005220A40A282823
:100070000230A200AA200030A40010302402013077
:1000800003180001003C03194D2801309F009920FE
:10009000C8308E005220A40A3D280230A200AA20B7
:1000A000812010280E0890006E308F0000000000A4
:1000B00000000000000000008F0B5628900B542811
:1000C00008008510FF3092001208003C013003192F
:1000D00000019203003C03196E28642809300310C4
:1000E00003188510031C85147528103E031C742802
:1000F000FF3E910C031D702885100A308E0052209F
:100100000800FE309100612001309100612008005C
:100110001E08003C03199828FE3091006120183019
:10012000910061200A308E0052201E089E0388280C
:1001300008001F08003C0319A928FE309100612027
:100140001C30910061200A308E0052201F089F034E
:10015000992808000030A3000A3023020130031858
:100160000001003C0319B92864308E005220A30A14
:04017000AC280800AF
:00000001FF
